:1000000050C500006BC5000069C500000C94D12FDD
:1000100065C5000063C5000061C500005FC5000044
:100020005DC500005BC500000C94AC2C0C94942DB5
:100030000C947F1B53C5000051C500004FC5000044
:100040004DC500004BC5000049C5000047C5000074
:1000500045C500000C94882C41C500003FC5000038
:100060003DC500003BC5000039C5000037C5000094
:1000700035C5000033C5000031C500002FC50000A4
:100080002DC500002BC5000029C5000027C50000B4
:1000900025C5000023C5000021C500001FC50000C4
:1000A0001DC500001BC5000019C500000501098021
:1000B000A101850319012AB700150126B700950192
:1000C00075108100C0050C0901A101850419012AE0
:1000D000A002150126A002950175108100C005013E
:1000E0000906A1018506050719E029E71500250184
:1000F0009508750181020507190029EF15002501F2
:1001000095F075018102050819012905950575010C
:100110009102950175039101C00660FF0961A1017B
:100120000962150026FF00952075088102096315F4
:100130000026FF00952075089102C005010906A15F
:1001400001050719E029E7150025019508750181CA
:10015000029501750881010507190029FF15002680
:10016000FF0095067508810005081901290515008D
:100170002501950575019102950175039101C0094D
:10018000025B00030100A0FA090400000103010161
:100190000009211101000122440007058103080024
:1001A00001090401000203000000092111010001FE
:1001B0002222000705820320000107050303200017
:1001C00001090402000103000000092111010001DE
:1001D000226D0007058403200001120100020000C7
:1001E0000008534601000100010200010C03430016
:1001F0006F0072006E0065000000100366006F0063
:100200006F007300740061006E00000004030904B5
:100210002B0014001A00080015001700E00004006D
:100220001600070009000A0000571D001B00060009
:1002300019000500000000000000E300777C2C009E
:100240002A00130012000C0018001C002F003300BD
:100250000F000E000D000B0029003800370036009B
:1002600010001100000000000000E600787C28006B
:1002700001001E001F0020002100220001001414B4
:100280002D005700340032000100351435022D14C2
:100290005500000000000000000001000100010006
:1002A000010027002600250024002300010032025F
:1002B000340264026400350001002E02341430144C
:1002C0002D022E00000000000000E600787C2800CF
:1002D000010000000000520000004A000100000080
:1002E000500051004F004D000100000000000000D0
:1002F00000000000000000000000010001000100FB
:1003000001005500610060005F0062005700240298
:100310005E005D005C003600560027025B005A005C
:10032000590037000000000000000100010001003A
:1003300001000000AC00AE00AB004278010045783F
:10034000477849784B7843780100467848784A786E
:100350004C780000000000000000010001000100D6
:10036000007C3D003C003B003A0046005009410043
:1003700040003F003E00000050094500440043009B
:100380004200000000000000000001000100010028
:1003900000AE00AF000101010101010101010202F3
:1003A0000202020202020203030303030303030423
:1003B00004040404040405050505050606060606EE
:1003C000070707070708080808090909090A0A0AA8
:1003D0000B0B0B0C0C0C0D0D0D0E0E0E0F0F0F104A
:1003E00010111111121213131414151516161717D4
:1003F000181819191A1A1B1B1C1D1D1E1E1F202040
:10040000212222232424252626272829292A2B2C89
:100410002D2D2E2F30313232333435363738393AAC
:100420003B3C3D3E3F404142434445464748494AA4
:100430004C4D4E4F50515354555658595A5B5D5E72
:100440005F616264656668696B6C6D6F707273750D
:1004500077787A7B7D7E8082838587888A8C8E8F71
:1004600091939596989A9C9EA0A2A3A5A7A9ABAD9F
:10047000AFB1B3B5B7BABCBEC0C2C4C6C9CBCDCF8D
:10048000D1D4D6D8DBDDDFE2E4E7E9EBEEF0F3F53B
:10049000F8FAFDFF00DA0281FFD9F1DB20A4A62ED5
:1004A000AF00A0C0D30000A1C8D30000AED580A883
:1004B0001F408D142000000000000000000000001C
:1004C000000000000000000000000000000000002C
:1004D00000000000000000000000FC020202028296
:1004E00042428202C242424202C2424242020202EC
:1004F00002FC0000000000000000FF000000000FF0
:1005000010100F001F020200001F02020000000076
:1005100000FF0000000000000000010202020202D1
:1005200002020202020202020202020202020202AB
:1005300002010000000000000000007C8282824472
:1005400000F8242224F800FE1212120C004C9292A1
:1005500092640000000000000000000000000000A5
:10056000000000000000000000000000000000008B
:1005700000000000000000000000FCFEFEFEFE7E09
:100580003E9E9E3E7EFE1E1EFEFE1E1EFEFEFEFECB
:10059000FEFC0000000000000000FFFFFFFFFFF076
:1005A000E0CFCFE0F0FFC0C0FCF9C0C0FFFFFFFF0D
:1005B000FFFF00000000000000000103030303032D
:1005C00003030303030303030303030303030303FB
:1005D00003010000000000000000007C82828244D1
:1005E00000F8242224F800FE1212120C004C929201
:1005F0009264000000000000000000000000000005
:1006000000000000000000000000000000000000EA
:10061000000000000000000000000C0A09894929C0
:10062000190981412111C93F0F010131190F84427C
:10063000211109050301C0A09088848281909894BB
:10064000929190F0FC838080E01CFC80808087F891
:10065000000000000000808080808080808080809A
:10066000808080808080808080808080808080808A
:100670008080808080800000000000000000FF017A
:10068000010101F1919191610101010101FF00005E
:100690000000000000000000000000000000FF80DB
:1006A0008080808F808182848880808080FF0000AD
:1006B0000000000000000000000000000000FF013A
:1006C000010101F1010101010101010101FF00002E
:1006D0000000000000000000000000000000FF809B
:1006E0008080808F888888888080808080FF00005C
:1006F0000000000000002020202061626364656625
:100700006768696A6B6C6D6E6F7071727374757601
:100710007778797A31323334353637383930524553
:1007200042545F2D3D5B5D5C233B27602C2E2F20C8
:100730002020000000000000000000000000000079
:1007400000000000000000000000000000000000A9
:100750000000000000007E0F00D4FFFFFFC7000074
:10076000007800000000000000002A2B2800000094
:100770000000000000000000000000000029000050
:1007800000002C1E3420212224342627252E362D2D
:100790003738271E1F202122232425263333362EC7
:1007A00037381F0405060708090A0B0C0D0E0F1039
:1007B0001112131415161718191A1B1C1D2F31307E
:1007C000232D350405060708090A0B0C0D0E0F1022
:1007D0001112131415161718191A1B1C1D2F31305E
:1007E000354C81422408102040808040201008248D
:1007F00042818142241008040201010204081024ED
:10080000428181C2E4F0F8FCFEFFFFFEFCF8F0E458
:10081000C2818143270F1F3F7FFFFF7F3F1F0F27AD
:100820004381010204081020408080402010080409
:1008300002010103070F1F3F7FFFFF7F3F1F0F07CD
:100840000301804020100804020101020408102066
:10085000408080C0E0F0F8FCFEFFFFFEFCF8F0E016
:10086000C08000000000000000005F0000000007E2
:1008700000070000147F147F1400242A7F2A12002E
:10088000231308646200364956205000000807030D
:100890000000001C224100000041221C00002A1C14
:1008A0007F1C2A0008083E08080000807030000005
:1008B0000808080808000000606000002010080414
:1008C00002003E5149453E0000427F40000072490F
:1008D000494946002141494D33001814127F100048
:1008E0002745454539003C4A494931004121110914
:1008F0000700364949493600464949291E0000008B
:1009000014000000004034000000000814224100E0
:10091000141414141400004122140800020159098F
:1009200006003E415D594E007C1211127C007F4949
:10093000494936003E41414122007F4141413E004C
:100940007F49494941007F09090901003E41415160
:1009500073007F0808087F0000417F4100002040AD
:10096000413F01007F08142241007F404040400089
:100970007F021C027F007F0408107F003E4141413E
:100980003E007F09090906003E4151215E007F09B2
:100990001929460026494949320003017F01030015
:1009A0003F4040403F001F2040201F003F40384054
:1009B0003F006314081463000304780403006159C2
:1009C000494D4300007F41414100020408102000CE
:1009D000004141417F0004020102040040404040C8
:1009E00040000003070800002054547840007F288E
:1009F00044443800384444442800384444287F00A4
:100A000038545454180000087E09020018A4A49C0D
:100A100078007F080404780000447D4000002040F6
:100A2000403D00007F102844000000417F4000004E
:100A30007C04780478007C0804047800384444443A
:100A40003800FC182424180018242418FC007C0802
:100A50000404080048545454240004043F4424006F
:100A60003C4040207C001C2040201C003C4030408A
:100A70003C004428102844004C9090907C00446432
:100A8000544C44000008364100000000770000008C
:100A90000041360800000201020402003C26232621
:100AA0003C0011241FBECFEFDAE0DEBFCDBF13E064
:100AB000A0E0B1E0ECEFF3E602C005900D92A032A9
:100AC000B107D9F728E0A0E2B3E001C01D92A83D2C
:100AD000B207E1F70E942F260C94943191CAEF924D
:100AE000FF920F931F93CF93DF93D22F4934D8F502
:100AF000C42FC695C695C695477020E2C29FD00107
:100B0000112470E06856784FA60FB71F60E070E0C0
:100B100028E030E0241B3109FC01E60FF71FE491C7
:100B20005D910E2F10E0FD0131977F01E02F042E23
:100B300001C0EE0F0A94EAF75E2BF70150834115CE
:100B400071F0C93061F0F801022E02C0F595E79509
:100B50000A94E2F75F965C915E2B5C935F976F5F00
:100B60007F4F6D17C8F2CDB7DEB7E6E00C941831B1
:100B70009C0191509F31B8F4832F817034FF0BC0DA
:100B80008295807F31FD806232FD806433FD806814
:100B9000FB010995089531FD826032FD846033FFC9
:100BA000F7CF8860F5CF80E0F3CF982F92959F70B4
:100BB00061F420E0982F892F8695869511F02E5F9D
:100BC000982F892F8695820F089524E0F4CF809383
:100BD0003D07089580933E07089521E001C0220F4C
:100BE0008A95EAF780913E07822BF4CF21E001C07D
:100BF000220F8A95EAF7822F809590913E078923EC
:100C0000E9CF292F983090F5863080F590E036E0D6
:100C1000239F800D911D112451E081FD54E080FD42
:100C2000550F82FD529523E0969587952A95E1F719
:100C3000FC01EE0FFF1FE80FF91FE25EF84F20E006
:100C400030E070E04191DF01CB01022E02C09695A9
:100C500087950A94E2F78695880B84278523842755
:100C60008E932F5F3F4F2330310561F70895292F71
:100C7000983070F5863060F590E036E0239F800D67
:100C8000911D1124682F677023E0969587952A950A
:100C9000E1F7FC01EE0FFF1FE80FF91FE25EF84FCE
:100CA00040E050E080E0219130E0062E02C0369511
:100CB00027950A94E2F72170042E01C0220F0A94AE
:100CC000EAF7822B4F5F5F4F4330510561F708957C
:100CD00080E0089590913E0721E030E0F90101C0E5
:100CE000EE0F8A95EAF7D90101C0AA0F6A95EAF7D3
:100CF000EA2B01C0220F4A95EAF7892F8E23E813C9
:100D000003C0892F822B66CF2095822F8923FBCFAA
:100D1000E091440790914307E91302C080E00895F1
:100D20009F0157E0E59FF0011124EB5BF84F5181E3
:100D3000561306C05081581303C05581541305C083
:100D40002F5F3F4FF901E770E7CF81E00895809171
:100D5000440720914307281301C008950196877026
:100D6000FACF90913F078095892380933F07282FE2
:100D7000277061F4891751F09091410792FF06C0E6
:100D800086958695869532DF10923F07089580916B
:100D90003A0790914207892B90913B079115C9F032
:100DA000892B90917401913021F49091400797FD27
:100DB00011C096E024E233E040E09150F901508107
:100DC0002F5F3F4F51114F5F9111F7CF411110929B
:100DD0003B0708959EE12CE233E0EECF8095982FFB
:100DE00080913A07892380933A070895803E9105C0
:100DF000D1F1C8F48133910509F481C048F48932F6
:100E0000910509F471C08A32910509F47FC00895F3
:100E100089339105E1F082389105C9F08533910558
:100E200009F45DC00895843E9105D1F148F4823EF5
:100E3000910531F1833E910541F181EE90E00895F5
:100E4000863E9105C1F1873E9105F1F1089520910B
:100E50004007237009F064C02091410723FF14C0AC
:100E600089E290E008952091400720FD45C030912F
:100E7000410730FF09C024FD24C083EE90E00895AF
:100E80002091400722FDF7CF08952091400722FDD1
:100E900044C03091410730FD43C024FFF5CF11C05D
:100EA0002091410721FFF0CF8091400784FD09C0C8
:100EB00087EE90E008952091400723FFE5CF24FFBF
:100EC000F7CF80E090E008952091400723FD2BC0EC
:100ED0003091410731FFE1CF84EE90E008952091F9
:100EE000400725FFD1CFBCCF2091400725FD1EC074
:100EF0002091410723FFC8CF89E390E00895209116
:100F0000400726FFC1CF8AE290E008952091400774
:100F100026FFBACF81E390E0089582EE90E0089535
:100F200080EE90E0089586EE90E0089585E390E0ED
:100F300008959091400792FF10C041E0282F24713E
:100F4000243009F040E031E0282F2871283009F0E2
:100F500030E0431711F02CE0822793FF10C041E0EE
:100F6000282F2471243109F040E031E0282F287126
:100F7000283109F030E0431711F02CE0822730913E
:100F8000410730FF10C051E0282F2171213009F0B6
:100F900050E041E0282F2871283009F040E0541734
:100FA00011F029E0822731FF10C041E0282F217184
:100FB000213109F040E031E0282F2871283109F073
:100FC00030E0431711F029E0822794FF02C083FD2F
:100FD000877E08950F931F93CF93DF9307DFEC0174
:100FE000D23508F04DC0D03508F0C3C0C03ED105A1
:100FF00030F5CD3CD10508F09AC0C83AD10578F457
:10100000C53AD10508F090C0C130D10599F1CE01A3
:101010000497813A910570F1C0E0D0E02BC0CE0179
:10102000885A91094B97C0F7C85AD0E0CC0FDD1F02
:10103000CC54DD4F0990D881C02DD4641BC0D0346E
:1010400090F4D03208F0A8C0C83ED10598F0CE0187
:1010500091509F3108F78D2F6CDF082F8C2F90E077
:10106000C5DE902B54C08C2F90E0C0DEDF70C82FFF
:10107000D92BD06ACE01DF91CF911F910F910895A6
:10108000C03882E5D807B8F5C03682E5D80708F041
:1010900056C0C03482E5D807C8F4C03282E5D8070C
:1010A00008F047C08C2F8695869520E2829FC0016C
:1010B0001124C37021E030E002C0220F331FCA9513
:1010C000E2F7E901C82BD92BDD68D4CF8C2F8695A8
:1010D0008695877020E2829FC0011124C37021E0B1
:1010E00030E002C0220F331FCA95E2F7E901C82B96
:1010F000D92BDC68BFCFC03C82E5D80750F48C2FD9
:101100008F71C03AD24580F5982F84EF906AEC0138
:10111000B1CFCE01805C9245809708F07DCFDC2F67
:10112000DF71C0EFD06AA6CFA497D064A3CFD065FB
:10113000A1CF8C2F8F71D82FC1EFD06A9BCF8C2F6E
:1011400086958695877020E2829FC0011124C37026
:1011500021E030E002C0220F331FCA95E2F7E90117
:10116000C82BD92BDA6886CFE4DEC0E0D82FD06256
:1011700081CF8C2F8F71DDDE93E0CC0FDD1F9A9530
:10118000E1F7DF70282F84FF04C090E1899F900170
:101190001124C22FD0696ECF8D2F8F71CADE082F18
:1011A0008C2F90E023DE902BEC01E1CF80E00895BE
:1011B000F894E82FE295EF70F0E041A18F7021E004
:1011C00001C0220F8A95EAF7922F9095942391A35C
:1011D00092A1822F892B82A378940895CF92DF92D7
:1011E000EF92FF921F93CF93DF93462F172FE82F95
:1011F000F0E0EC56FC4F71110CC0E4918E2F7E2F65
:101200006E2FDF91CF911F91FF90EF90DF90CF90E5
:101210000895F491EF2F86E0689FE00111242FEFED
:1012200030E0CE01B9010E94DC30DB01CA01880F39
:10123000991F65E56A9FA0016B9F500D1124841BC7
:10124000482F440F480FC901811B9109F89F700175
:10125000F99FF00C11248F2D149FB0011124672FDA
:1012600070E06901C61AD70AB601F69F6001F79FC0
:10127000D00C1124A330B10549F1B901641B7109E7
:10128000AB01149FB001159F700D1124672F70E002
:10129000261B370BF29FA001F39F500D1124752FD1
:1012A000CC3FD34050F4A130B105A1F0129709F022
:1012B000A7CFEF2D852F7F2FA3CFA430B10569F0E5
:1012C000169709F49DCF7F2D8D2D9ACF7D2DEF2D73
:1012D0008F2F96CF7F2FED2D93CFE52F7F2DF8CF3A
:1012E000982F8091ED06811529F081E09B3108F05F
:1012F00080E0089581E09633FACF9C0180E090E091
:10130000269F020E811D369F800D911D1124830F93
:10131000911D089540910C0150910D0125E038E098
:10132000429FC001439F900D529F900D1124875EF4
:10133000994C80930C0190930D01890F0895982F7B
:10134000E82F96FDE0958E2F8F7096FD8F5FE695C6
:10135000E695E695E670F0E0E659FD4F2181289F7D
:10136000202D812D112422952F708295807F282B8E
:101370008081820F97FD8195805808951F93CF93A8
:10138000DF93EB01182F822F8695D9DF805887FDD8
:101390008195880F282F219F020E20E0211D112406
:1013A000822FBE01DF91CF911F910895622F089582
:1013B000E42FF0E0EE0FFF1FE853FE4F6081621B49
:1013C00008950F931F93022F50E0FA01EE0FFF1FB5
:1013D000E856FE4FE1A9E052E7FDE195440F551FA5
:1013E00048535E4FDA012C91201B310B2E0F620FF8
:1013F0001F910F9108950F931F93A02FB0E0FD014F
:10140000EE0FFF1FE856FE4F01A90052110B2003FB
:10141000F001219FF00D1124AA0FBB1FA853BE4F4E
:101420002C912057330B4203D001439FB00D112460
:101430009F012A0F3B1F12F421583F4F220F232FE9
:10144000221F330B620F1F910F9108959091270473
:10145000982B9093270408953091ED06311521F0D3
:101460008B3191052CF008958B31910514F04B9739
:10147000C6C108951F93CF93DF93C82FD0E0FE011C
:10148000EC5CFD4F808190910A01892389F042DF55
:10149000182F40DF20E8829FC0011124792F715856
:1014A000612F8091C2069ADE472F282FCE01D4DF0C
:1014B000DF91CF911F910895FF920F931F93CF93C8
:1014C000DF93182F062FF42EC0E0D0E02F2D402FF1
:1014D000612FCE01C1DF2196C633D105B9F7CDB753
:1014E000DEB7E5E00C941931982F990F990F890F09
:1014F000982F9B5F973308F096E32091ED0621111A
:1015000004C08B3128F48BE108959C3108F09BE1F5
:101510000895EF92FF920F931F93CF93DF937C0177
:1015200080910901E1DFC82F192F6091C3066695EC
:10153000669521E0620F08F46FEF8091230490918B
:101540002404DBDE082FD0E0812FC11730F0C8DE85
:10155000CDB7DEB7E6E00C941831FE01EC5CFD4F30
:10156000808190910A01892379F06091C006709181
:10157000C1068091C206202F4C2FF70109952EDE5F
:10158000472F282FCE0168DF2196DECF9091BF062E
:1015900021E092279093BF061092080157CF8091C7
:1015A000BF06837011F4109208018091BF068C7FF2
:1015B00081608093BF0608958091BF06837011F00B
:1015C000109208018091BF068C7F8093BF0608951A
:1015D0009091BF06937091F0811589F0893088F45D
:1015E0008F73880F880F982F2091BF062370922B3E
:1015F0009093BF0610920801862F28CF089581E0AE
:10160000F0CF88E0EECF8091BF06869586958F5FFC
:10161000893008F081E061E0DBCF8091BF068695DC
:101620008695815009F488E061E0D2CF9091BF06A1
:10163000937059F08093C0066093C106493708F053
:1016400048E74093C206822F01CF0895EFEBF6E002
:10165000818190E021E0438162810896E7CFEFEB42
:10166000F6E0818121E0438162818850990BDECFD1
:10167000EFEBF6E0628120E1620F08F46FEF818109
:1016800021E0438190E0D2CFEFEBF6E0628120E1F0
:10169000621B08F460E0818121E0438190E0C6CFC5
:1016A000EFEBF6E0438120E1420F08F44FEF818138
:1016B00021E0628190E0BACFEFEBF6E0438120E1D8
:1016C000421B08F440E0818121E0628190E0AECFCE
:1016D0002091C30630E1230F08F42FEF2093C306B7
:1016E00081E0B4CE2091C30630E1231B08F420E052
:1016F0002093C30681E0AACEE091C406EF3F69F0D3
:10170000E53069F0E23069F4EF5FF0E0EC56FE4F4F
:1017100080818093C40681E099CEE0E0F5CFE1E0DE
:10172000F3CFE0E0F2CFE091C406EF3F91F0E53077
:1017300071F0E23019F0E1110EC0E3E0E150F0E0A9
:10174000EC56FE4F80818093C40681E07FCEE1E0BD
:10175000F5CFE3E0F4CFE0E0F2CF20912804382F7A
:101760003203C0011124923014F080E090E0825ADC
:101770009B4F80933C0490933D0408950F931F93D7
:10178000CF93DF93A0913C04B0913D049D012E5571
:101790003440620F731F613042E0740710F060E064
:1017A00072E04091600650916106FC0101E010E09A
:1017B0002617370748F04093600650936106DF9183
:1017C000CF911F910F91089584919D91981789F061
:1017D000ED018A93C901C5E096958795CA95E1F711
:1017E000E80102C0CC0FDD1F8A95E2F7CE014C2B39
:1017F000592B2F5F3F4F3196DBCF539A0895FC0151
:10180000EE0FFF1FE80FF91FE458FC4F6183408380
:1018100022830895FC01AC014C5F5F4F8FEF61E3C1
:101820009191892728E030E0982F990F87FF09C010
:10183000892F862721503040B9F7E417F50781F743
:101840000895892FF7CF811144C0E5E6F3E020E049
:1018500030E047E0429FC001439F900D1124DC011E
:10186000A659BC4F5C9153FF06C05681511103C06D
:101870008B599C4F08952F5F3F4F3796233031058A
:1018800049F7611531F180916A0383FF1CC0809193
:10189000710383FF1BC08091780383FD1AC082E02F
:1018A00090E027E0289FF001299FF00D1124CF013F
:1018B0008B599C4FDC0116961C92E659FC4F2081F7
:1018C00028602083089580E090E0EBCF81E090E0F5
:1018D000E8CF80E090E008954115510511F0FA013C
:1018E000099508958091EC06811103C08091BE0690
:1018F0000895E0911407F0911507309739F00190A1
:10190000F081E02D309711F00995089580E0089559
:10191000A3E0B0E0EEE8FCE00C940031209163031A
:101920003091640328173907B1F0809363039093D3
:101930006403E0911407F0911507309761F000847B
:10194000F185E02D309739F023E029838A839B834A
:10195000CE01019609952396E2E00C941C31A3E098
:10196000B0E0E5EBFCE00C94003120916103309194
:10197000620328173907B1F08093610390936203E3
:10198000E0911407F0911507309761F00084F1851C
:10199000E02D309739F024E029838A839B83CE01A0
:1019A000019609952396E2E00C941C319091740104
:1019B000913099F0A4E2B3E0EFEF90E02C91821720
:1019C00059F01196EF3F19F4211101C0E92F9F5FE3
:1019D0009630A1F7EF3FC1F408959091400797FF2B
:1019E000E9CFE82FE695E695E695803FA8F7F0E089
:1019F000E65DFC4F877021E001C0220F8A95EAF76F
:101A00008281822B82830895FE2FFF0FFF0BEE5DF4
:101A1000FC4FF8CF90917401913021F490914007E0
:101A200097FD0CC0E4E2F3E09191891302C0DF015D
:101A30001E9293E0EA32F907B9F70895E82FE69588
:101A4000E695E695803FC8F7F0E0E65DFC4F9DEF38
:101A500081FD97EF80FF959582FD92958281892384
:101A6000828308958091730108952FB7F89460914F
:101A70005D0370915E0380915F03909160032FBFBF
:101A800008958091EC06811539F0EFDF462F572F2E
:101A9000BC01CB01BA010895E8DFDC01CB01409124
:101AA000EE065091EF066091F0067091F106480F36
:101AB000591F6A1F7B1FEDCF87E797E780930008C8
:101AC0009093010888E19AE00FB6F894A895809366
:101AD00060000FBE90936000FFCF0895FC0120913D
:101AE0005303309154032617370748F061157105E9
:101AF00029F49091E8009E779093E8009B0190E094
:101B00002115310541F4911106C08091E80082FF52
:101B100032C080E0089580916A068115C1F1853058
:101B2000C1F18091E80083FD30C08091E80082FD22
:101B3000ECCF8091E80080FFE3CF8091F3004091EB
:101B4000F200582F2115310519F04830510558F091
:101B500091E04830510509F090E04091E8004E775F
:101B60004093E800CDCF81918093F100215031095D
:101B70004F5F5F4FE7CF80916A06811541F0853056
:101B800041F08091E80083FFC0CF81E0089582E0BA
:101B9000089583E00895982F9093E900891771F0D4
:101BA0007091EC002091ED005091F00021FD09C0F2
:101BB0009F5F973089F78093E9000895762F242F4F
:101BC00050E03091EB003E7F3093EB003091ED0020
:101BD0003D7F3093ED003091EB0031603093EB00AE
:101BE0007093EC002093ED005093F0002091EE00F4
:101BF00027FDDECF089580914D0387FF13C08091AC
:101C0000E80082FF06C08091E8008B778093E800AF
:101C1000089580916A068111F2CF089580916A0635
:101C20008115D9F38091E80080FFF8CF8091E8001A
:101C30008E77ECCF2091E4003091E50095E6A90184
:101C40002091EC00822F817020FF06C08091E80077
:101C500080FF06C080E008952091E80022FD1AC0B0
:101C600080916A06811589F0853089F08091EB00BA
:101C700085FD0FC02091E4003091E5004217530725
:101C8000F9F29150E1F684E0089582E0089583E04E
:101C9000089581E00895CF93DF93C8EDD0E0888167
:101CA0008F7E8883E7EDF0E080818160808384E02F
:101CB00082BF81E080934C0388818E7F8883E2EE2F
:101CC00010821092DA00A1EEB0E01C9288818F772A
:101CD000888388818068888388818F7D888319BC08
:101CE00010926A0610924B0310922A0410924A0333
:101CF000A0EE8C918B7F8C9388818160888342E0F9
:101D000060E080E048DFA1EEB0E08C918E7F8C93A4
:101D1000E2EEF0E080818160808380818860808352
:101D2000E0EE80818E7F8083888180618883DF916F
:101D3000CF910895E8EDF0E080818E7F808310924E
:101D4000E2001092DA001092E100A0EEB0E08C9177
:101D500081608C9380818F77808319BCA7ED8C91F3
:101D60008E7F8C9380818F7E808310924C030895A8
:101D7000A0E0B0E0EEEBFEE00C94F630D82E8091BF
:101D800081018D1549F00091960710919707011573
:101D9000110539F4D0928101CDB7DEB7ECE00C9497
:101DA00012318D2D0E94D505B82E9091950780E0B7
:101DB000891781F3F8012081B21609F455C08F5FAD
:101DC0000B5F1F4FF5CFF8010180F281E02DEE0D82
:101DD000FF1D2081822F81568A31B8F42052205273
:101DE000330B46E0429FC001439F900D112425E034
:101DF000492D62E08E59974F0E946F058FEFE81AC8
:101E0000F80A892D865F982E65C0203240F720E2BF
:101E1000E6CFED120FC0A814B90401F582E398E0F3
:101E200020E14C2F60E10E946F058FEFE81AF80A5D
:101E3000C85F6CC0C7010197A816B90691F082E08F
:101E400098E0AE14BF0461F31F3F29F082EE97E0E3
:101E5000AE14BF042CF382EF97E0E2CF82E298E069
:101E6000DFCF82E198E0DCCF81819281892B09F478
:101E700091CFD0919407D11509F48CCFE8E9F7E020
:101E800080E491E011920197E9F7F801A181B28114
:101E9000FD0101900020E9F73197EA1BAE2ECD2E0F
:101EA000C3944AE04E9F402D1124425080E590E0BB
:101EB0009C01241B3109A90155954795942E2C2D81
:101EC000220F220F220F821B910995958795C82F0B
:101ED000E12CF12CEA1408F476CFE4E8F7E010E006
:101EE000A081B181109719F08C918B1529F0329651
:101EF0001F5F1D13F5CF1FEFE12CF12CA12EB12E8A
:101F0000BB0CBB088D2F8150990B4C01EC1408F0D1
:101F100041CFE1107ECF82E598E0111509F480CF22
:101F200082E498E07DCFA0E0B0E0E9E9FFE00C9426
:101F3000F8307C016B015A018091D3060AE010E071
:101F40008A3010F001E010E0C1E0D0E0B601C70136
:101F5000F5010995811115C021960C171D078CF00C
:101F6000CC9F9001CD9F300D300D112480E090E08A
:101F700045E34A95F1F70000019682179307C1F7F0
:101F8000E5CFCDB7DEB7EAE00C9414313BB1377F33
:101F90002BB128604FB7F8948CE793E0FC010196D1
:101FA000508168E02BB9000000C057FF3BB9550FC6
:101FB000000000C000C000C03BB900C06A9591F7A6
:101FC00054E08E31950751F74FBF8FE594E00197AC
:101FD000F1F700C0000008950F931F93CF93DF9394
:101FE000EB018A0190916A06943059F58093E900DB
:101FF0008FEF9091E80095FD06C095ED9A95F1F769
:1020000000008150B1F78091E80085FF1AC012DE10
:10201000811112C08091E80085FD06C08091E80022
:102020008E778093E800F3CF88818093F100015090
:10203000104011F02196EECF8091E8008E778093CA
:10204000E800DF91CF911F910F910895603229F43C
:1020500040E250E0BC0182E0BFCF0895CF93DF9310
:10206000EC0148E050E0BC0181E0B6DF88E0FE0111
:10207000A5E5B3E001900D928A95E1F7DF91CF914C
:10208000089540E250E0BC0184E0A6CF43E050E078
:10209000BC0184E0A1CF9091410792FB222720F957
:1020A000281779F080FB92F99093410760914007DF
:1020B0007091410784E090E00E94903182E00C949E
:1020C000B10608951F93CF93DF93122F8630E0F46B
:1020D0006830D0F44630C0F4C42FD0E0CC0FDD1F00
:1020E0002CE0629FC00DD11D112490E6899FC00D88
:1020F000D11D1124632FCE0189960E947631612F64
:10210000CE018A960E947631DF91CF911F9108957A
:10211000AF92BF92CF92DF92FF920F931F93CF9314
:10212000DF93A12CB12CC0E06501D0E018C021E004
:1021300030E0C43020F4F801859195919C014F2D39
:102140006D2F8C2FBFDFF3940E5F1F4F8F2D8630C6
:1021500071F7DF5F86E0C80ED11CD83039F08601F8
:10216000000F111F005F1D4FF12CE1CFCF5F80E307
:10217000A80EB11CC630C1F6DF91CF911F910F910F
:10218000FF90DF90CF90BF90AF9008958091740141
:10219000813069F58091400787FF29C00E94C706FA
:1021A00080932B0340E250E064EF76E08AE293E014
:1021B0000E943431892BD1F080E2EAE2F3E0A4EF0F
:1021C000B6E001900D928A95E1F7E0911407F09145
:1021D0001507309759F00480F581E02D309731F0E4
:1021E00086E080932A038AE293E0099508950E948D
:1021F000C7068093220348E050E066E177E082E280
:1022000093E00E943431892B89F388E0E2E2F3E025
:10221000A6E1B7E001900D928A95E1F7E0911407ED
:10222000F0911507309711F30280F381E02D30977C
:10223000E9F282E293E0D9CF811531F090913A072B
:10224000982B90933A07A2CF0895811531F0909181
:102250004207982B9093420799CF0895811519F062
:102260000E94EE0693CF0895811539F080959091E4
:10227000420789238093420789CF0895CF93C82FBF
:102280008115C1F08450813A70F5809174018130DC
:1022900021F48091400787FD0FC0E4E2F3E08081E4
:1022A000C817E9F0319683E0EA32F807C1F78C2FBE
:1022B0007DDB6CDFCF910895EC2FE695E695E695F2
:1022C000F0E0E65DFC4F828190E04C2F477021E00A
:1022D00001C0220F4A95EAF78223892B41F38C2F04
:1022E00099DB54DFE4CF8C2F805E883060F4C770B8
:1022F00081E001C0880FCA95EAF7C0913A07C82B60
:10230000C0933A07D6CF8C2F855A833028F48C2F70
:102310008452990BFDDACECFC85ACB3158F6EC2F48
:10232000F0E0EE0FFF1FE651FD4F8081918117DB3A
:10233000C1CFCF93DF93EC01805E9109089720F025
:1023400065E271E1209711F46CE171E1CE010E9428
:10235000B8058C2F93DFDF91CF910895CF93DF9352
:10236000EC018A81823039F4FB0182819381E1DFC3
:102370008D8182608D83DF91CF910895FB018081F3
:102380009181D7CF811511F1982F9450913A10F483
:1023900041DBFCCE982F905E983058F4982F81E066
:1023A00091FD84E090FD880F92FD82950E94EE06DB
:1023B000F0CF982F955A933018F480E090E0A8CA97
:1023C000885A8B3118F480E090E0C9CA0895CF9301
:1023D000DF93EC01D7DFCE01805E9109089720F0F2
:1023E00064E371E1209711F46EE271E1CE010E9485
:1023F000B805DF91CF910895FC018281813029F4E5
:10240000FB0180819181E3CF08958230E9F7FB01E0
:1024100082819381F8CF1F93CF93DF93182FEB0125
:102420002DDF209731F4812FADDFDF91CF911F9108
:1024300008958FE99FE00197F1F700C00000219710
:10244000F0CF10923A0780917401813099F4809115
:10245000400787FF0FC0ECE2F3E08EE111928A950E
:10246000E9F780E090E054DA80E090E078DA1092CA
:1024700042078CCEE4E2F3E086E0F0CFE2DF88E1D1
:102480009AE00FB6F894A895809360000FBE9093E1
:102490006000FFCFAAE2B0E0E0E5F2E10C94FF308B
:1024A0008DE493E0FC0101962091F100208323E06C
:1024B00085359207B9F780914E03893009F457C0EA
:1024C000C8F4823009F4B3C0833009F483C081308A
:1024D00081F18091E80083FFE7C080914D039091E6
:1024E0004E039A3008F0E0C0E92FF0E0EA56FE4CC7
:1024F0000C9427318A3009F48AC08B3051F78091CF
:102500004D03813231F78091510390915203892B11
:1025100001F78091E800877F8093E8006CDB81E021
:1025200090914F03911101C080E08093740189DF85
:10253000D0CF80914D03813A61F68091E800877F8A
:102540008093E8008091510390915203892B59F0B8
:1025500060E080E090E070E0C1DA8091E8008B7785
:102560008093E800B6CF68E085E593E0F4CF8091F2
:102570004D03813209F0ADCF809151039091520308
:102580008D7F892B09F0A5CF8091E800877F80930C
:10259000E8008091E80082FF18C02091F30080914C
:1025A000F200922F029731F48091F100813011F006
:1025B000863021F48091F100809373018091E800CE
:1025C0008B778093E80017DB84CF80916A068111B6
:1025D000E0CF7FCF80914D03813A09F07ACF80918F
:1025E000510390915203892B09F073CF8091E80039
:1025F000877F8093E8008091E80080FFFCCF809186
:1026000074018093F1008091E8008E77DACF809199
:102610004D03813209F05DCF8091E800877F809380
:10262000E800E9DA809150038093720152CF8091E3
:102630004D03813A09F04DCF8091E800877F809368
:10264000E8008091E80080FFFCCF80917201D9CF33
:10265000803889F0823841F5809151038F7087303E
:1026600018F58093E9008091EB0085FB882780F9BD
:102670001092E90006C080912A04880F90914A03C5
:10268000892B9091E800977F9093E8008093F10068
:102690001092F1008091E8008E7723C0811116C05E
:1026A00080914F03813009F18091E80083FF0AC0D7
:1026B0008091E800877F8093E8008091EB00806242
:1026C0008093EB00AA96E3E00C941B31823061F713
:1026D00080914F03811579F01092E9008091E80014
:1026E000877F8093E80087DADFCF933009F080E0BE
:1026F00080932A04F1CF809151038F70282F2150AD
:10270000263090F68093E9002091EB0020FFE4CF83
:10271000933031F48091EB0080628093EB00DCCF4A
:102720009091EB0090619093EB0021E001C0220FAB
:102730008A95EAF72093EA001092EA008091EB0074
:102740008860EBCF8111B0CF80914F038F77182F26
:102750008091E3008078812B8093E3008091E800F2
:10276000877F8093E80047DA8091E80080FFFCCF04
:102770008091E30080688093E30083E0111101C041
:1027800082E080936A0690CF8058823008F08CCF28
:1027900080914F03909150038C3D23E0920789F57F
:1027A00083E08A838AE289834FB7F894DE01139627
:1027B00020E03EE051E2E32FF0E050935700849197
:1027C00020FF03C082958F703F5F8F708A30B8F012
:1027D000895C8D931D922F5F243169F74FBF8091E3
:1027E000E800877F8093E8006AE270E0CE010196FE
:1027F00075D98091E8008B778093E80055CF805D94
:10280000E8CF292F30E02330310509F44DC078F5A9
:102810002130310509F47CC08BE590E0EFE7F1E071
:102820002230310509F040CF2091E800277F209326
:10283000E80020915303309154038217930708F462
:102840009C0140E02115310509F067C0411165C0C8
:102850008091E80082FDCDCF80916A06811549F212
:10286000853039F28091E80083FFF2CFC2CF8091AA
:1028700051039091520321323105D9F122323105B1
:1028800009F012CF8330910508F00ECFFC01EE0F56
:10289000FF1FE857FE4F0190F081E02D8B579E4FB0
:1028A000DC018C9190E011C0282F30E0813089F05C
:1028B00022303105B1F0232B09F0F6CEECE0F2E046
:1028C000E4918E2F90E0ECE0F2E0009709F4ECCE7A
:1028D000ABCFEAEFF1E0E4918E2F90E0EAEFF1E088
:1028E000F4CFECEEF1E0E4918E2F90E0ECEEF1E02D
:1028F000ECCF8330910508F0D7CE880F991FFC01EB
:10290000E257FE4F0190F081E02D89E090E08CCFFE
:1029100082E190E0EAEDF1E087CF80916A068115CF
:1029200009F467CF853009F464CF8091E80083FD16
:1029300060CF8091E80082FD8BCF8091E80080FF1E
:1029400081CF4091F3008091F200942F2115310541
:1029500019F08830910550F041E0089709F040E007
:102960008091E8008E778093E8006CCF449140938B
:10297000F1003196215031090196E8CF803809F0F5
:1029800093CE8091E800877F8093E80080914B038D
:102990008093F1007FCE811187CE80914F03182F55
:1029A000823008F081CE8091E800877F8093E80034
:1029B00010934B0320D91115D9F084E080936A0657
:1029C00042E061EC81E0E7D842E261EC84E0E3D8E8
:1029D00042E261EC82E0DFD842E260EC83E0DBD8E7
:1029E00080916A06843051F482E0809375015CCE58
:1029F0008091E30087FDE1CF81E0E0CF81E0F5CF7A
:102A0000CF93DF93EB01FC01448155816085718593
:102A1000CE010E946C0C9B81909580914207892386
:102A2000809342078C810E94EE06B0DB87E019920A
:102A30008A95E9F7DF91CF9108950F931F93CF9374
:102A4000DF938C01EB018D8181FD17C082608D8346
:102A5000809142079B81892B8093420780913A079E
:102A60009C81892B80933A0791DBF8014281538145
:102A700060857185CE010E946C0C10923407109213
:102A800035078D8180FD03C0BE01C801B9DFDF912C
:102A9000CF911F910F910895CF92DF92EF92FF9205
:102AA0001F93CF93DF9300D000D0CDB7DEB7C09097
:102AB0008406D0908506E0908606F09087060E94F6
:102AC000350DDC01CB018C199D09AE09BF0911E060
:102AD00084369105A105B10578F10E94410DDC0114
:102AE000CB010296A11DB11D89839A83AB83BC8360
:102AF00080913B0190913C018C56994F20913A0175
:102B0000422F50E0253008F044E09E012F5F3F4FF8
:102B1000B9010E94413183E090E00E946E30182F8D
:102B2000811551F00E94350D6093840670938506DF
:102B30008093860690938706812F0F900F900F90B9
:102B40000F90DF91CF911F91FF90EF90DF90CF908A
:102B50000895A0E0B0E0EFEAF5E10C94F630B82E6D
:102B6000EB01A42E4901C880D980EA80FB800E9435
:102B7000350DDC01CB018C199D09AE09BF098436E6
:102B80009105A105B10510F4A11421F1EB2CFB2C4A
:102B9000FF0CFF089B2D88E09802F0011124EE5DE8
:102BA000FE4F818192818C56994F2081422F50E0B7
:102BB0000217110508F4A801B4010E944131C701B0
:102BC0000E946E30811539F00E94350D688379833B
:102BD0008A839B8381E0CDB7DEB7ECE00C941231A1
:102BE0000F931F9341E09091A10680913E079813A7
:102BF00001C040E001E010E02EE337E060E876E05D
:102C000084E0A7DF811571F041E09091A2068091E8
:102C10003D07981301C040E02DE337E06CE776E014
:102C200085E097DF1F910F910895A1E0B0E0EBE1FF
:102C3000F6E10C94FE3080916F0689832091AD06F9
:102C400090E041E02817190609F440E08D019E014B
:102C50002F5F3F4F60E776E088E07BDF2196E4E07E
:102C60000C941A31CF92DF92FF920F931F93CF9360
:102C7000DF93F82E6B01EA01A801B901CE010E9491
:102C8000343141E0892B09F440E09E01B6018F2DDB
:102C900060DFDF91CF911F910F91FF90DF90CF9078
:102CA00008950F931F9304E010E029E936E0AC018A
:102CB00068E876E082E0D6DF1F910F910895A1E0E9
:102CC000B0E0E5E6F6E10C94FE300E94720C8983D8
:102CD00001E010E023EA36E0AE014F5F5F4F68E7A6
:102CE00076E086E0BFDF2196E4E00C941A31A9E09B
:102CF000B0E0EDE7F6E10C94FE3088E0EFEBF6E0B3
:102D00009E012F5F3F4FD90101900D928A95E1F707
:102D1000198609E010E024EA36E0CE010196AC0104
:102D200064E776E087E09EDF2996E4E00C941A31B0
:102D3000ACE0B0E0EEE9F6E10C94FE308091CF0615
:102D40009091D006A091D106B091D20689839A8342
:102D5000AB83BC838091CB069091CC06A091CD062D
:102D6000B091CE068D839E83AF83B8878091C706CE
:102D70009091C806A091C906B091CA0689879A8722
:102D8000AB87BC870CE010E02EEA36E0AE014F5F67
:102D90005F4F6BE676E089E065DF2C96E4E00C940B
:102DA0001A31AF92BF92CF92DF92EF92FF921F93B0
:102DB000CF93DF9300D000D00F92CDB7DEB75B0189
:102DC00080E090E00E946E30182F811509F462C0F7
:102DD00080912501482F50E0811141E0609126014A
:102DE000709127016C56794FCE0105960E944131B2
:102DF000C0909006D0909106E0909206F0909306D5
:102E00000E94350DDC01CB018C199D09AE09BF096B
:102E100084369105A105B10538F485E996E00E9454
:102E20000A0C9D818917B1F181E090E00E946E301B
:102E30008115F1F180912D01482F50E0853008F087
:102E400044E060912E0170912F016C56794FCE01B4
:102E500001960E94413185E996E00E940A0C9D810D
:102E6000891326C00E94350D6093900670939106D9
:102E7000809392069093930689819A81AB81BC815D
:102E800080938C0690938D06A0938E06B0938F0648
:102E900081E00FC08091950690919606A0919706CB
:102EA000B091980689839A83AB83BC831111E4CFD8
:102EB00080E040918C0650918D0660918E06709155
:102EC0008F06F50140835183628373830F900F90C7
:102ED0000F900F900F90DF91CF911F91FF90EF9087
:102EE000DF90CF90BF90AF9008950F931F93CF9333
:102EF000DF93863008F56830F8F44630E8F4C42FE4
:102F0000D0E0CC0FDD1F9CE0699FC00DD11D1124C6
:102F100090E6899FC00DD11D1124CE0189960E9493
:102F20005A31082FCE018A960E945A31902FDF9194
:102F3000CF911F910F91089580E090E0F8CF462F38
:102F4000783030F4663020F4863010F4672FCDCF1F
:102F500080E090E00895CF92DF92FF920F931F934D
:102F6000CF93DF936C0100913E0780913D07082BC2
:102F7000C5E0D0E010E0C8010C2E02C09595879501
:102F80000A94E2F780FD0CC02197A8F7F12C8F2D51
:102F9000DF91CF911F910F91FF90DF90CF90089517
:102FA000FC2EB6018C2FCBDF0E94EA07019761F35C
:102FB000EECF1F93CF93DF93FC012581C081D18198
:102FC000CE01211579F0611569F0C5DF182F682F42
:102FD000CE010E940106BE01812FB1DFDF91CF91AA
:102FE0001F9108950E943706182FF5CFCF93DF93D6
:102FF000EC01B1DFBE01A3DF0E94EA07DF91CF91B0
:103000000895FC012481211599F080819181EEDFE2
:10301000282F92959F70963099F060F4925F9F7080
:10302000923030F4203FB1F038F481E0283E38F09F
:1030300080E008959A5FF3CF81E0243FC9F70895B7
:1030400091E0213F09F090E081E0283E08F080E027
:10305000892B089581E00895673921E07207810581
:10306000910528F4CB0187599D4F0C945A3180E08B
:103070000895CF92DF92EF92FF92CF93DF93EC010E
:10308000C880D980EA80FB80B601C701E5DF9FEFE9
:10309000C91AD90AE90AF90AC882D982EA82FB82E6
:1030A000DF91CF91FF90EF90DF90CF90089585E270
:1030B00090E00E945A31863269F486E290E00E94E4
:1030C0005A31863039F487E290E00E945A3191E01B
:1030D000803109F090E0892F8170089580E090E0C0
:1030E0000E946231833E9E4F09F4E1CF80E0089553
:1030F00048E050E067E170E08FEB96E00E946731B6
:1031000010922704089581E18093BF068091820187
:1031100090918301A09184018093C0069093C10691
:10312000A093C2068FE78093C3068FEF8093C406F7
:10313000DFCFA0E0B0E0EFE9F8E10C94FA300E94B4
:10314000410DAB01BC0140931E0450931F048093BA
:103150002004709321041091220480910801823090
:1031600009F4D5C1D0F4811120C010920901409317
:1031700023045093240460932504709326048091C3
:10318000BF06837021F08091BF0686958695809357
:10319000220481E08093080103C0833009F4C1C197
:1031A000CDB7DEB7E8E00C94163180910701181313
:1031B00025C09091BF0693702091060130E081E018
:1031C0009217130609F480E080930B018091C406E6
:1031D00090910A01981739F080930A0140E060E06D
:1031E00080E00E945C0A193058F4E12FE150E83089
:1031F000E8F4F0E0E056FE4C0C94273181E0E4CF97
:103200001F3F09F454C180E0909109019F5F9093A2
:1032100009018111C5CF82E08093080180910B01E3
:103220008111BECF1111BCCF83E0B4CF80910B01CF
:10323000811549F340E060E080E00E945C0AE3CF42
:10324000809109010E94740AC82F092F6091C0065D
:103250007091C1068091C2060E94EE08F62EE72EFC
:10326000D82ED0E00C1709F020F4802F0E947009AE
:10327000CBCFFE01EC5CFD4F808190910A01892348
:1032800031F02D2D4E2D6F2DCE010E942C0A21964E
:10329000E9CF8EEB99E00E94890AB6CF86ED99E0DE
:1032A000FACF88ED99E0F7CF81EE99E0F4CF8091E5
:1032B00009010E94740AC82F092F6091C306669500
:1032C00080912304909124040E947D09D82ED0E09F
:1032D000CE01880F991F88569E4F7C010C1729F24A
:1032E00020F2FE01EC5CFD4F808190910A01892360
:1032F00009F451C0F70140A94057550B81A98052EC
:10330000990B449F9001459F300D300D1124889FEB
:10331000A001899F500D500D1124240F351F822FBD
:103320002230310520F19FEF213E8EE1380740F435
:10333000C901E5E096958795EA95E1F7982F985FA2
:1033400061E0462F490F5527551F55954795842F06
:10335000449FF001459FF00DF00D11242E173F07FB
:10336000F8F4942F9150961760F7862F815090E0D3
:10337000BC01660F771F680F791F759567956D0DF6
:103380007091C1068091C2060E94EE08472F282F37
:10339000CE010E942C0A219682E0E80EF11C9ECFFD
:1033A0004F3F29F3642F6F5FDECF809109010E94A8
:1033B000740AC82FF92E6091C306669566958091B0
:1033C0002304909124040E947D09E82E805C0E94D1
:1033D0009F098058D82E8E2D0E949F098058C82E94
:1033E000D0E0CF1510F08F2D41CFFE01EC5CFD4FEA
:1033F000808190910A01892391F06091C0067091BB
:10340000C1068091C2060C2F2C2D4D2D0E94FB0968
:103410000E94EE08472F282FCE010E942C0A2196E9
:10342000E0CFC0910901C1111FC06091C30620E126
:10343000620F08F46FEF80912304909124040E949E
:103440007D0965E070E00E94DC30892B69F40E9400
:103450008A0926E3829FA0011124852F880F880BFB
:1034600050930401809305018C2F0E94740AEC0193
:1034700090910B01911117C0209104013091050129
:103480002817310590F02D17310578F4822F0E940E
:103490003A0A87E3809304011092050106C08C2F3D
:1034A0000E943A0ACF5FCD17D0F38D2FDFCE9091D7
:1034B0002404A0912504B0912604892F9A2FAB2FC4
:1034C000A69597958795A69597958795837090E093
:1034D000A0E0B0E082309105A105B10589F083300C
:1034E0009105A105B10579F040E060E010979040AA
:1034F000814059F464E180E00E945C0A82E04ACE97
:1035000044E160E0F8CF44E164E184E1F5CF109359
:1035100007018091BF068370809306010E94C60F49
:1035200083CE809127048111E3DDE0902304F090A5
:10353000240400912504109126048091EC06811545
:1035400079F00E94350D6E197F09800B910B653063
:1035500071058105910508F423CE1092080120CE53
:103560000E94410DF0CFA0E1B0E0E9EBFAE10C944C
:10357000F230FE013196DF0180E11D928A95E9F774
:103580000AE110E099E6A92E92E0B92E612C712C87
:10359000230153944A189E2E8F2E6201730181E1FC
:1035A00048165104610471041CF080E1C82ED12C2E
:1035B000A601B501892D982D0E946731AC0CBD1C68
:1035C0000D2C000C00084C185D08600870080150B4
:1035D000104019F76096E0E10C940E316FEF85E230
:1035E00090E00E9476316FEF86E290E00E947631A3
:1035F0006FEF87E290E00E94763160E088E290E031
:103600000E9476310E948810AEDF66E285E290E08B
:103610000E94763166E086E290E00E94763160E1B9
:1036200087E290E00C94763163EE7EEF80E090E0EC
:103630000E94903160E082E090E00E94763181E06B
:1036400080933D0761E083E090E00E94763160E086
:1036500074E184E090E00E94903155DDBFDF60E0CE
:1036600070E0AB018FE090E00E94883160E070E094
:10367000AB0183E190E00E9488313ACDAB0124E6B2
:1036800030E0BC0188E70E94A52E9C0181E0232B3D
:1036900009F080E00895809168068115F1F00E949C
:1036A000350DDC01CB01805A9541AF4FBF4F809360
:1036B000620690936306A0936406B09365068091BA
:1036C0006F0681110AC062E070E082E993E0D6DF04
:1036D000811519F081E080936F0608958091680646
:1036E000811561F080916F06811541F062E070E014
:1036F00080E993E0C3DF811110926F0608951F9255
:103700001FB61F9211248F939F93AF93BF93809105
:103710002904811113C080915D0390915E03A091F3
:103720005F03B09160034196A11DB11D80935D03BD
:1037300090935E03A0935F03B0936003BF91AF913A
:103740009F918F911F901FBE1F9018952FB7F894CF
:1037500080915D0390915E03A0915F03B09160033F
:103760002FBF0895CF93DF93EC01F0DF8C1B9D0BEF
:10377000DF91CF910895ACE0B0E0E1ECFBE10C9477
:10378000F730FE013196DF0188E01D928A95E9F756
:103790008AEAC82E82E0D82E7F01AE2E9F2C04EB41
:1037A00012E0F60181916F018F3F09F43DC0F8945A
:1037B000E82FE295EF70F0E021A18F7041E001C0A9
:1037C000440F8A95EAF7922F942B91A392A1842F0C
:1037D0008095892382A3789400C0EEEAF2E031E07C
:1037E000B12C21912F3F79F0A22FA295AF70A05E4E
:1037F000B0E08C9190E02F7002C0959587952A9546
:10380000E2F780FFAEC080E0B82A330F0E171F0723
:1038100041F7F60182918F3F11F00E94D80880EAAB
:103820008A95F1F7F701B0828FEFE81AF80A8EEA6D
:10383000C81682E0D80609F0B4CF48E050E06A2DFF
:10384000792D84EE96E00E943431009749F028E00B
:10385000EA2DF92DA4EEB6E001900D922A95E1F73C
:103860000091E30610E00552194F892B09F47BC043
:1038700081E08093DA066ADF8093D8069093D906B8
:103880008091EC06811509F4C6C07E0189E0E80E3E
:10389000F11CF70184E011928A95E9F78091D30633
:1038A0008A3008F083C041ED56E1B701C8010E949B
:1038B000930F811509F49EC041E556E1B701C80197
:1038C0000E94930F811509F495C04CE455E1B701AE
:1038D000C8010E94930F811509F48CC040EF55E197
:1038E000B701C8010E94930F811509F483C04FE509
:1038F00056E1B701C8010E94930F811509F47AC0FF
:1039000047E756E1B701C8010E94930F811509F4FA
:1039100071C045E156E1B701C8010E94930F8115BE
:1039200009F468C048E956E1B701C8010E94930F45
:10393000811509F45FC01092D3068091D70690E0FC
:1039400044E050E0B7018552994F0E94343121E0A4
:103950002093D606892B09F03FC02C96EBE00C94FF
:103960001331832F51CF8091DA06811509F488CF66
:10397000E090D806F090D906E9DE8E199F090597E8
:1039800008F47ECF44E050E064EE76E0C8010E9487
:103990003431892B41F084E0E4EEF6E0D801019067
:1039A0000D928A95E1F71092DA066ACFC090D4069C
:1039B000D090D506CBDE8C199D09843F914008F04C
:1039C00072CF8091D606811541F2F70184E0119201
:1039D0008A95E9F71092D606E091D706F0E0E55215
:1039E000F94F89859A85AB85BC8580839183A283B5
:1039F000B383B3CF8091D3068F3F31F4A7DE80939A
:103A0000D4069093D506DDCF8F5F8093D3068A309E
:103A100008F493CFF3CFE090D706F12CC70185527D
:103A2000994F7C01F80180819181A281B3818093BB
:103A3000950690939606A0939706B093980685E90D
:103A400096E00E940A0C80939406809199069091CA
:103A50009A06A0919B06B0919C06F7018083918302
:103A6000A283B383C0909D06D0909E06E0909F06EF
:103A7000F090A0068091BA069091BB06A091BC067A
:103A8000B091BD06C816D906EA06FB06B1F0C09291
:103A9000BA06D092BB06E092BC06F092BD060E9428
:103AA000350DC61AD70AE80AF90AC092EE06D09276
:103AB000EF06E092F006F092F1068091A106809365
:103AC0003E078091A20680933D078091A3068093D4
:103AD000BE0688E0E4EAF6E0AFEBB6E001900D92B6
:103AE0008A95E1F78091AD06811591F1D4DD809141
:103AF000B6069091B706A091B806B091B90640916C
:103B0000B2065091B3066091B4067091B50600916B
:103B1000AE061091AF062091B0063091B106009329
:103B2000CF061093D0062093D1063093D20640934F
:103B3000CB065093CC066093CD067093CE0680934F
:103B4000C7069093C806A093C906B093CA0605CFCE
:103B5000C5DDCDCFFF920F931F93CF93DF93C62F79
:103B6000D42FF22E8115A9F060933807EFDD8093F2
:103B70007A0390937B0381E0C1FD84E0C0FD880F50
:103B8000C2FD82950E941C11CDB7DEB7E5E00C9412
:103B9000193180913807681333C000917A0310916E
:103BA0007B03D4DD801B910B883C910548F51D2FCC
:103BB000105ECD17A1F0C77001E0802F01C0880F03
:103BC000CA95EAF70E942E11183048F48D2F87709D
:103BD00001C0000F8A95EAF7802F0E941C1160E057
:103BE00070E08F2D0E940B1281E0D1FD84E0D0FDAA
:103BF000880FD2FD8295183038F60E942E11C4CF5E
:103C000081E0C1FD84E0C0FD880FC2FD8295F5CF43
:103C1000A4E0B0E0EEE0FEE10C94F5307C01FC01A4
:103C20008481811509F448C161E0C701C2D96C01E2
:103C3000F70185818115D1F0009134071091350786
:103C40000115110599F0C016D10689F027E7A22EBB
:103C500021E0B22E011511F0A12CB12C60E0802FD3
:103C60000E94230CFC01892B09F040C08601F7015A
:103C70008581811509F452C0918190933307908119
:103C80009093320790E2909376010093300710935F
:103C90003107980130523032C8F59681903130F0BA
:103CA000E02FF0E0ED33F10508F48BC0F7019581CA
:103CB000911509F47EC510923807980130572332C8
:103CC000310508F084C584E090E00E946231809361
:103CD000400790934107F801E150F047E232F105C7
:103CE00008F098C1E855FE4C0C942731858184601A
:103CF0008583C082D182BF01C5010E941D1510922B
:103D0000420761E0C70155D98C01B1CF9801305409
:103D1000303108F046C09681903110F6312F37557A
:103D200009F051C1A02EB12C0111B7C0682F80E05D
:103D30000E94230C6C01892B09F4AFC0F701858127
:103D4000F601958180FB90F99583811509F41AC1DC
:103D5000FDDC8093360790933707F60182818F5FF1
:103D600082838091420790913A07892B83838091C7
:103D70003B078483409177015091780160917F01E6
:103D800070918001C6010E946C0CF601858181FD55
:103D900003C0A12C97E5B92EA0923407B092350745
:103DA00085CF980131503F3108F47ACF9801205ADD
:103DB00032452032310508F479CF0D33110538F43E
:103DC000F801EA50F94FE491E0937601A7CF98010A
:103DD00037572038310508F0A1CF003108F05DC019
:103DE00066E971E080E090E037D9811156C0A12CDE
:103DF000B12C450101111FC089829A82AB82BC821D
:103E00008E010F5F1F4FC80134D9B02EA12E813013
:103E100008F443C009F06BC0C8012BD98130F1F41C
:103E2000C80127D960E570E0893311F060E070E0E7
:103E30000E940B12E8CF87E9881681E09806A1045A
:103E4000B10459F1B401C50107D99FEF891A990A44
:103E5000A90AB90A8111EFCF0150CCCF823029F4E1
:103E6000C80107D90E943E11CECF833029F4C80182
:103E700000D90E94C211C7CF843069F4C801F9D8B3
:103E8000C12CD12C282F2053330B2A303105C0F000
:103E9000C114D10411F58111B6CF80913F0787700D
:103EA00059F0F7018581811539F08091410782FF32
:103EB00003C082E00E94B1062496EDE00C9411311B
:103EC0004AE04C9DC0014D9D900D1124280F391FD3
:103ED00069018B2D9A2DCDD8D5CFEFE9FFE0319731
:103EE000F1F700C0000091E0C91AD108D1CFE82F46
:103EF000F0E0EE59F84F9491792E282F26952695CB
:103F0000269530E0F901EE5AF84FC4908770D12C15
:103F1000082E02C0D594C7940A94E2F7F901EE5B2B
:103F2000F84FA490B12C082E02C0B594A7940A941F
:103F3000E2F72E5C384FF9018490912C02C09594E1
:103F400087948A95E2F7C0FE03C081EE0E943E117D
:103F5000A0FE03C086EE0E943E1160E070E0872D57
:103F60000E940B12A0FE03C086EE0E94C211C0FE8A
:103F700003C081EE0E94C21180FE45CF60E070E078
:103F80008CE256CF40917D0150917E0160917F017E
:103F900070918001C6010E946C0CF601858181FF41
:103FA00085CEB60187E791E00E9400158091340725
:103FB000909135078115974509F078CE1092340716
:103FC0001092350773CEF801E851FC47E730F10550
:103FD00008F06CCEE653FE4C0C94273126E241EEFD
:103FE00061EEB8DD5ACF27E245EE65EEFACF26E264
:103FF00041EE60EEF6CF27E245EE64EEF2CF26E228
:1040000041EE62EEEECF27E245EE66EEEACF28E221
:1040100041E0EBCF80914007816080934007609141
:1040200040077091410784E090E00E9490310E9427
:10403000211233CF80914107886080934107EFCFF1
:10404000809140078260E9CF809140078460E5CF8E
:10405000809140078860E1CF809141078160EDCF7A
:10406000809141078260E9CF809140078061D5CF80
:10407000809140078062D1CF809140078064CDCF8E
:104080000E942112809140078068C7CF809140072D
:104090008C60C3CF809141078360CFCF8091400770
:1040A0008E7FBBCF80914107877FC7CF809140072C
:1040B0008D7FB3CF809140078B7FAFCF809140073A
:1040C000877FABCF809141078E7FB7CF809141072B
:1040D0008D7FB3CF809140078F7E9FCF8091400727
:1040E0008F7D9BCF809140078F7B97CF0E942112BD
:1040F000809140078F7791CF80914007837F8DCF4C
:10410000809141078C7F99CF90914007892F8B7FB9
:1041100092FF8460877F92FF88607FCF8091410704
:10412000982F909590FB80F990FB81F986CF909124
:104130004007892F8F7B96FF80646FCF0E942112EA
:1041400090914007892F97FB87F9805866CF61E0EF
:104150008EE090E00E94763162CF60E0F9CF9091DE
:104160004007892F8F7E94FF806157CF9091400741
:10417000892F8E7F90FF816050CF90914107892FCA
:10418000877F93FF886059CF89E233C389E21CC3DC
:1041900080913A078272F801E054F847EF30F10558
:1041A00008F059C0EF52FE4C0C9427318272F8018E
:1041B000E052F847EB30F10508F04DC0E052FE4CFC
:1041C0000C94273181E00E94C60A67CE811511F157
:1041D0000E940D0B62CE811511F10E942F0B5DCE56
:1041E000811511F10E94440B58CE811511F10E94E6
:1041F0005C0B53CE811511F10E94720B4ECE0E94C2
:10420000CF0A81E00E94260A48CE0E94DC0AF9CF3C
:104210008115F1F20E94030B40CE8115F1F20E944C
:10422000260B3BCE8115F1F20E94380B36CE81155C
:10423000F1F20E94500B31CE8115F1F20E94680B11
:104240002CCE811529F00E94930B27CE8115D9F32E
:104250000E947C0B22CE07378CE71807F1F0083755
:104260008CE7180729F19801205E3245203231058C
:1042700020F5911134C00F7181E090E002C0880FE9
:10428000991F0A95E2F78C01682F83E090E00E9465
:104290007631802F0E94E70500CE81E0911551F024
:1042A0000E94ED0543E062E081E00E946A06F5CDE0
:1042B00082E0F4CF0E94F605F5CF911581F10B3520
:1042C0008CE7180711F10C358CE7180799F00A35BF
:1042D0008CE71807C1F001308CE71807F1F00330C4
:1042E0008CE71807A1F001151C47C9F40E942112A0
:1042F0000E945C0D80914107002482FF0394802D71
:104300000E944B10CACD81E0FBCF80E0F9CF6FEF68
:104310007FEF80E090E00E9490310E943E12F70112
:1043200000811181911509F45BC0C8010E94AB178F
:10433000D82E682FC8010E940106B8018D2D0E9459
:104340009F170E94EA07182FA92EF701B580D68083
:10435000D2948FE0D82280913F07877001F1CB2C57
:10436000B114F1F0892F807F803461F0812F805E5D
:104370008830A8F0892F807E803221F4123078F0C6
:10438000D11469F08091410782FF09C082E00E9448
:10439000B10680913F078770CC24C3948111C12C52
:1043A0008A2D82958F70883009F409C1C0F5843058
:1043B000E0F4823008F444C00A2D0F708A2D807F0B
:1043C000803211F00295007F113008F472C009F4B8
:1043D000BBC0B11409F4C6C0D11409F488C048C0E8
:1043E000C8010E943706D82EA8CF09F4CCC0C1144A
:1043F00009F414C180913F0780FD10C1F7011582B7
:104400008695869586950E94ED05C70101DC809111
:104410003F078695869586950E94F605FFC08930F0
:1044200009F448C18A5F8F70823008F7123F09F0A3
:1044300053C18A2D8F71B1104CC10E94ED05ECC0A3
:104440000A2D0F708A2D803110F00295007FB11473
:10445000B9F0011569F0812F805E883010F01111DC
:1044600009C080913A07802B80933A070E94C610BA
:10447000812F2FC080914207802B80934207F6CF77
:10448000812F0E94C211011509F4B1CF812F805EE6
:10449000883010F0111104C0802F0E94EE0606C073
:1044A0000095809142078023809342070E94C610A6
:1044B0009ECF8091410782FD16C0B11469F00115AD
:1044C00039F080913A07802B80933A070E94C610FA
:1044D00080E00E943E118BCF80E00E94C211011546
:1044E00009F485CFD9CFB114A9F0D11004C0802F21
:1044F0000E941C117CCF8D2D813009F078CF8091E6
:104500003B07902F9823091709F471CF802B8093D4
:104510003B076DCFD1106BCF802F0E942E11909151
:104520003B07802F892329F0802F80958923809352
:104530003B0780913C07902F982309F458CF0095B2
:10454000082300933C0753CF8D2DB11421F0863002
:1045500008F04DCFCCCF853008F049CF802F0E9496
:104560002E1145CFD114D1F3193349F48FEF97EEC3
:1045700023E0815090402040E1F700C00000812FEF
:104580000E94C21134CF8A2D869586958370813022
:1045900060F009F02CCF812F9A2D9370B11002C0DA
:1045A00080E090E00E94AF0C22CF812F9A2D937073
:1045B000B11002C080E090E00E94880C18CF8A2DD4
:1045C0008370E1F5B11028C0812F829586958770A0
:1045D000880F880F412F4F70082E01C0440F0A9496
:1045E000EAF7212F207114FF06C02FE001C0220F2F
:1045F0008A95EAF720958A2D869586958370982F5F
:104600008230A1F08330B9F080913D07913059F0AC
:10461000242B82230E94E7050E94720C60E0C701F0
:104620000E94D91749CC842B822BF4CF242B809164
:104630003D078227EFCF822F842BECCFB11459F1A5
:10464000A0FEEACF812F829586958770880F880F0C
:10465000412F4F70082E01C0440F0A94EAF7212F12
:10466000207114FF06C02FE001C0220F8A95EAF7DF
:1046700020958A2D869586958370982F823091F0AB
:104680008330A9F080913E07913049F0242B82239A
:104690000E94EA05C1CF823008F4BECFD3CF842B6D
:1046A000822BF6CF242B80913E078227F1CF822FD9
:1046B000842BEECF8A2D8F70082FB11431F00E9419
:1046C000ED05812F0E941C11A7CF812F0E942E1172
:1046D000802F0E94F605A0CF70F4103FC9F0113F63
:1046E00091F0B11409F451C0D11409F44BC0812FD9
:1046F0000E943E1191CF133FF9F0143F91F7909132
:10470000410792FD26C08A2D8F71B11411F395CE09
:104710008D2DB11479F0853008F07ECF8A2D8F7100
:10472000282F81E001C0880F2A95EAF790913E0773
:104730008927AECF8630F0CF80E0B11409F4A8CF3E
:104740008A2D8F71982F81E001C0880F9A95EAF722
:104750009FCFB11461F08A2D8F7192FF6ECE982F8A
:10476000990F990F990F936090933F0766CE81E060
:104770000E94B1068D2D823008F44ECF82E00E9457
:10478000B1064ACF8A2D8F7158CED11479F01933E2
:1047900049F48FEF97EE23E0815090402040E1F7FD
:1047A00000C00000812F0E94C21136CF8A2D8F7168
:1047B00090CF06318CE7180709F0EACC80913907D1
:1047C000811509F4E3CC85E30E940A0D14C08091A1
:1047D0003A0706312CE7120709F0E8CC8A7A91E013
:1047E000811101C090E090933907811509F4CCCC78
:1047F00085E30E94D60C0E94C6104FCB80918307A0
:10480000803170F480918207811551F0E091440766
:104810002091430730917E0740917D072E1301C000
:104820000895BF0187E0E89FF0011124DF01AB5B31
:10483000B84F14968C911497811551F111968C9163
:104840001197831325C08C91841322C015968C91E7
:10485000159781111DC012968D919D91A0917F0792
:10486000B09180078A1B9B0B883C910588F480914E
:1048700083078F70806180938307E55BF84F8081A9
:104880008F70806180838DE797E0C2D90C94A70672
:104890006F5F7F4FFB01E770C1CFADE0B0E0E3E5B4
:1048A000F4E20C94F5308C0186E0F801DE011896F4
:1048B00001900D928A95E1F7F801F58084819DE7DA
:1048C000892E97E0992E70908107711017C081157D
:1048D00091F0F11409F40EC1C8010E94011881156C
:1048E00009F408C187E0F801ADE7B7E001900D9247
:1048F0008A95E1F783DFFF24F39455C0D080A2802E
:10490000B380C090820720917F0730918007A50176
:10491000421B530BC11409F4BDC0483C510508F0BB
:1049200076C0811541F380917E079180E0908307E6
:104930009E2D903108F057C0981214C080917D07C9
:104940008D1110C0F11049C08E2D8F708061809341
:1049500083078DE797E05CD980918307F801868310
:10496000F12C21C0F11039C040E0692D8D2D0E943D
:10497000880640E0692D8D2D0E948806F82E811151
:10498000EFCF888599850E94F617292F22952F70E1
:10499000903470F49F70223098F09115A9F0F801CE
:1049A0009681903188F48F2D2D96EDE00C94113185
:1049B0002A5F2F70223060F0C8012AD9FC2CF3CF77
:1049C000911511F0811579F3805E883060F3F4CF92
:1049D000803F48F3815F8330F9CF80918307816006
:1049E00080938307BDCF981237C080917D078D11CA
:1049F00033C0F11031C0E682C8010AD987E0F8015E
:104A0000ADE7B7E001900D928A95E1F774CFE090A1
:104A100083079E2D903148F48DE797E0F9D8F40193
:104A200087E011928A95E9F79BCF811509F463CF4E
:104A300090917E07818198130FC080917D078D1121
:104A40000BC0F11009C0E682C801E2D8F40187E08A
:104A500011928A95E9F74FCFC8010E94011881157C
:104A600009F448C0F11409F445C08E2D803208F4D1
:104A700039CF80917D0790917E0789839A83AB829D
:104A8000BC827D821E82809183078F83CE01019636
:104A9000BFD828CF483C510508F0C1CF811509F493
:104AA0002ACFF11439F190917E078181981318C0B3
:104AB00080917D078D1114C08091830780FD9ECF6A
:104AC000803108F49BCF8683807F803F09F494CFA8
:104AD0008681982F907F905F8F70892B86838CCFF3
:104AE000C8010E9401188111FDCE80918307816069
:104AF00080938307C8018CD8FECEABE1B0E0E3E839
:104B0000F5E20C94FE304E8B5F8B688F798F8A8F25
:104B1000192F9B8F9111109242071D8A86E0FE018A
:104B20007696DE011F9601900D928A95E1F70A8D27
:104B3000011561F00B8B1C8B61E0CE010F960E947A
:104B4000D91761E0CE010F960E94D9170B8B1C8BF1
:104B500087E0FE013F96DE01189601900D928A953E
:104B6000E1F7CE01089699DE81112EC0209143070E
:104B70003091440787E0AE01485F5F4FFA0147502C
:104B80005109DA0101900D928A95E1F78C85811522
:104B9000D9F0822F90E08395877090E0AC013417B4
:104BA0001506E1F097E0929FD0011124AB5BB84F5E
:104BB0009E012F5F3F4FF90101900D929A95E1F709
:104BC000409343070E94A7068091440790914307B2
:104BD000891311C06B96E4E00C941A310E942112E3
:104BE0001092430710924407EDE7F7E087E0119237
:104BF0008A95E9F7E9CF27E0829FC00111248B5BFA
:104C0000984F4BDE811531F3809144079091450711
:104C10000196877080934407D7CFA6E0B0E0E3E128
:104C2000F6E20C94FE300E94A61B8C018091F206E5
:104C30009091F3068017910771F019821A820E94F1
:104C4000A61BBC0149815A8180E090E056DF0093A9
:104C5000F2061093F3062696E4E00C941A31CDB7D1
:104C6000DEB7A4970FB6F894DEBF0FBECDBF85B7F1
:104C7000806885BF85B7806885BF84B7877F84BF1C
:104C80000FB6F894A89580916000886180936000C9
:104C9000109260000FBE80E890E00FB6F894809309
:104CA0006100909361000FBE81E08093750186EDF5
:104CB00098E080932003909321030E949A0E0E9413
:104CC0004B0E8091E20084608093E20078948091A2
:104CD0006A06811599F08091E9001091EC008F70BF
:104CE00010FB112717F9182B1092E9008091E800AA
:104CF00083FD0E944A121F701093E90082E084BD78
:104D000093E095BD9AEF97BD80936E001092EE06EA
:104D10001092EF061092F0061092F1060E945718BA
:104D2000811102C00E94EE1A8091D80080618093A8
:104D3000D8008AE18A95F1F700C08091D900182F38
:104D4000117080FD04C00E949A0E10926A061093A2
:104D5000EC060E946E18811102C00E94141B8EE0A6
:104D600090E00E945A31811529F060E08EE090E0D9
:104D70000E9476318EE090E00E945A3191E08111DC
:104D800001C090E09093ED0690930E018091EC06A7
:104D900081110E948D2F8091ED0691E08927880F67
:104DA000880F8093E30694E0981B9093D7066AEAF5
:104DB000E62E62E0F62E0EEA12E0F70181917F0105
:104DC0008F3F11F00E94D8080E151F05B1F75EEA5B
:104DD000E52E52E0F52E04EB12E0F70181917F0100
:104DE0008F3F11F00E94D8080E151F05B1F7EBEDAB
:104DF000F6E088E011928A95E9F7E4EEF6E088E0C3
:104E000011928A95E9F70E946E18811102C00E94E2
:104E1000141B82E090E00E945A318093330484E0B6
:104E200090E00E94623180934007909341070E9476
:104E3000BB1B8FEF96E721E0815090402040E1F7C7
:104E400000C000000E94BB1BE091ED0611E0E127CD
:104E5000EE0FEE0FF0E0E552F94F808181FF08C0C0
:104E60006FEF7FEF80E090E00E9490310E945C0D38
:104E700083E090E00E945A310E94E7050E94FD0BFA
:104E80001093270448E050E067E170E08FEB96E074
:104E90000E944A31109227048091BF06843010F49A
:104EA0000E94831883E080935E0680E2809328044A
:104EB000CFD66BE070E08BEA94E00E943E1B811538
:104EC000E9F180915E0665E070E081FD0FC186EA40
:104ED00094E00E943E1B811589F16DE070E084E949
:104EE00094E00E943E1B811549F10E94350DDC01C2
:104EF000CB01805A9541AF4FBF4F8093620690938C
:104F00006306A0936406B0936506EEE5F4E0DF0166
:104F100080E092E01D920197E9F7E0933C04F09362
:104F20003D048FEF9FEF809360069093610681E0D0
:104F30008093680680936F0610925F068091EC065E
:104F4000811101C0EDD78CE892E080939607909391
:104F5000970784E080939507ACE8B2E020E01396D1
:104F60008C911397811501F12830F0F4822F90E095
:104F7000FC01EE0FFF1FEC57F84F8F01009761F017
:104F8000F801529142918F01FA01348114966C918B
:104F90001497631708F4ADC0880F991F8C57984F6A
:104FA000FC01A083B1832F5F159682E0A03AB80779
:104FB000B1F62093940780913E070E94B80E8FE0CF
:104FC00091E0809314079093150791E0C92ED12C9E
:104FD00080916A06853069F400E110E482E1F82EE0
:104FE00080916A06853009F489C00E9421120E94CE
:104FF000720C0E94BB1BA4E3AA2EA4E0BA2EBBED48
:105000008B2EB6E09B2EF401D5019D9180812CE37F
:1050100034E02A173B0709F4CCC031969817A9F35E
:105020002090EC06FBE2EF2EF4E0FF2E712CF40151
:1050300061904F01F50141905F01461409F441C0B0
:10504000462400E010E055245394842D852189F1F5
:10505000362C35202114F9F0F701808190E096017B
:10506000002E01C0220F0A94EAF78223892B99F4BB
:1050700009837A820E94A61B8B839C8381E08D83A7
:1050800091E0311001C090E09E8349815A816B818B
:105090007C818D8132DD31100CC08C2D002E01C041
:1050A000880F0A94EAF7982F9095F7018081892359
:1050B0008083550C0F5F1F4F0630110531F6F50147
:1050C000629273948FEFE81AF80A872D883009F0FE
:1050D000AECF0E94410D6093CF067093D0068093AF
:1050E000D1069093D206BB24B39467C081EA94E0C2
:1050F000F0CE0197F8014283538340CF80916A0636
:10510000843039F10E9499180E946E1B1092290474
:1051100088E190E00FB6F894A895809360000FBEE8
:105120001093600083B7817F846083BF83B7816001
:1051300083BF7894889583B78E7F83BF0FB6F8942A
:10514000A895809160008861809360001092600053
:105150000FBE0E94BB1BEBEDF6E0ABE2B4E080E0DB
:1051600021912D9391E0211101C090E0892B96E0CF
:10517000E33EF907A9F7811509F432CF80912A049B
:10518000811509F42DCF09BDF9BC09B400FEFDCF8E
:105190008091D8008F7D8093D8008091E00082605C
:1051A0008093E0008091E00081FDFCCF0E942112FD
:1051B00017CF981335CF31DDB12C8091EC068115D6
:1051C00031F1E0903407F0903507E114F104F9F083
:1051D00000913607109137070E94A61B801B910B88
:1051E000893C9105A0F007E711E0E11411F000E01F
:1051F00010E060E08E2D0E94230C009741F0FC012E
:10520000258122FD04C0BC01C8010E941D150E9419
:10521000991880916806811509F47CC00091660692
:10522000109167060E94A61B801B910B819708F4C2
:105230004FC00E94A61B809366069093670680E08D
:105240000E94AD0B80913E070E94B80E8091ED0642
:10525000811509F4B1C080E00E94AD0B60E670E0FA
:1052600086E196E00E94BE0B83E00E94AD0BE091C8
:105270003C04F0913D04CF018E559440AF014E5156
:105280005340413022E0520710F040E052E02091BC
:105290006006309161067F01A8E9B7E084179507A1
:1052A00008F46EC020936006309361068DE00E9482
:1052B000AD0B60E470E086EB96E00E94BE0B8FE0E1
:1052C0000E94AD0B60E270E086EB94E00E94BE0BA2
:1052D0008091600690916106892B09F08EC08091C3
:1052E0006F068115B9F00E94350D0091620610918C
:1052F00063062091640630916506DC01CB01801BBA
:10530000910BA20BB30B8F3F9F4FAF4FBF4710F4D2
:105310000E946E1BB1100E944B1B0E94720C909158
:105320006906891721F0809369060E94350D8091E6
:105330006A06843009F04CCE83E08093E9008091C6
:10534000E80082FF45CE8091E80090E085FF06C02E
:105350000E941A0E811509F427C191E08091E8009E
:105360008B778093E800911509F432CE8981E82F7C
:10537000E150E33108F042C1F0E0E551FE4C67C76F
:105380001D91F70161917F011617A1F0BF016150D6
:105390007109FB011083BC01E5E076956795EA95FC
:1053A000E1F7F60102C0EE0FFF1F6A95E2F7BF01B9
:1053B0002E2B372B019672CF0E94720C06E715E058
:1053C00081FD02C006ED14E080E00E94AD0B60E6B6
:1053D00070E086E196E00E94BE0B84E00E94AD0B77
:1053E00060EA70E0C8010E94BE0B8DE00E94AD0B28
:1053F00060E470E086E796E069CF809168068115E9
:1054000009F46DCF80915F06811169CF0E944B1B1B
:1054100031E1E32EF12C20916006309161062115D7
:10542000310509F45CCFEA9411F459CFF3948F2D30
:1054300090E026010F2C02C0440C551C0A94E2F7A0
:10544000A20142235323452B89F320915E0620FDC0
:1054500042C09695879596958795482F282F9F2D22
:105460009295990F9076392F315E842F90931D017C
:105470008093200130931E012093210124E630E027
:1054800047E050E06BE171E088E715D4892B09F023
:1054900026CF80E2F89E3001112480915E0680FDC7
:1054A00023C0A301425A5B4F04E610E020E230E043
:1054B00060E488E790D4892B09F011CF4094509490
:1054C0008091600690916106842195218093600609
:1054D00090936106A0CF9F2D990F990F990F392FA7
:1054E000395F80E023E0C2CFEEE3F4E080E2119286
:1054F0008A95E9F784EA92E089A39AA300EA12E088
:1055000068EA72E0A9A1BAA1ED91A9A3BAA3D80152
:105510008D918D01282F260D372D311D2BA33CA3F6
:10552000F0E0E25CFB4F20E030E097E0892E821A49
:10553000AC2C022E01C0AA0C0A94EAF78BA19CA104
:10554000825A9B4F1C0190E0D1018D911D018A214F
:10555000482D491B477050E0A82F042E01C0AA0F08
:105560000A94EAF7519541955109477001C0869513
:105570004A95EAF78A2B4081842B80839F5F98307D
:1055800019F72F5F3F4F31962830310571F689A109
:105590009AA16817790709F0B5CF04E610E020E278
:1055A00030E04EE354E084CF80E2E82EF12C8E010F
:1055B0000F5F1F4F8091E80085FD0AC08091E800D1
:1055C0008B778093E8000E941A0E811599F3C5CE5F
:1055D0008091F100F801808381E0E81AF10809F474
:1055E000BCCEE6CF1A828CE08B8319C08A818330CF
:1055F00081F138F4813029F1823051F08FEF8983C5
:105600000EC08430D9F71B821C821D821E8207C007
:1056100088E290E04FD61B821C821D828E83E0912F
:105620001407F0911507309709F4D2CC0284F38562
:10563000E02D309709F4CCCC60E2CE0101960995BB
:10564000C7CC0E94350D09D66B837C838D839E83E6
:10565000E6CF8B8190E0FE01349688309105FCF610
:1056600011920196FACF8A81823031F0853031F67D
:1056700080E00E94C60AD3CF6B817C818D819E81A0
:10568000ECD588E290E032D6CACF4C816B818A811A
:105690000E9475179827892798278D839E83BFCFEF
:1056A0002D813E813227232732274C816B818A81CD
:1056B0000E946210B4CF0E948810B1CF9A819330BB
:1056C00009F09CCF883009F439C0893009F462C0F0
:1056D0008B81833061F158F4813091F0823009F090
:1056E0009ECF8C8181111CC00E94DC0A98CF84302F
:1056F00009F095CF8C8120E04091C2066D810CC0ED
:105700004C8128E7429F040E40E0411D1124809106
:10571000C00620E06091C10690E00E94160B7FCF8A
:105720000E94CF0A60E08C810E94E80A78CF8C81C9
:105730008093C30680E00E94260A71CF8B8183305C
:1057400031F170F48130B1F0823009F068CF80918E
:10575000BF06982F9370C9F0869586958C835FCF8E
:10576000843009F05CCF8091C0068C838091C106A3
:105770008D8355CF8091C2062FEF829FC0011124E7
:1057800068E770E019D56C834ACF80E0E7CF80915D
:10579000C306E4CF0E94781842CF80E18A833FCFCE
:1057A00081E08A8387E920CF8A809B80982489249E
:1057B0009824A12CB12C8E010F5F1F4FEC80E00EBE
:1057C000F12EF11C0E151F0509F429CF87E9881663
:1057D00081E09806A104B10470F4C40187599D4F7B
:1057E00069D5F80184830F5F1F4F8FEF881A980ADD
:1057F000A80AB80AE7CF80E0F4CFFC808A809B80BB
:10580000982489249824A12CB12C8E010F5F1F4F5E
:10581000250132014F1451046104710408F0FFCED8
:1058200087E9881681E09806A104B10430F4F801F4
:105830006481C40187599D4F59D58FEF481A580A82
:10584000680A780A8FEF881A980AA80AB80A0F5FC0
:105850001F4FE0CF0E94B31AE2CE86E09FCFFC80BC
:105860008A809B80982489249824A12CB12C25011E
:1058700032018E010B5F1F4F4F14510461047104FC
:1058800008F0CDCE80E4881682E09806A104B10429
:1058900088F4C40189960ED5F80181938F018FEFAA
:1058A000481A580A680A780A8FEF881A980AA80ACC
:1058B000B80AE2CF80E0F0CFFC808A809B809824F9
:1058C00089249824A12CB12C8E010F5F1F4F250134
:1058D00032014F1451046104710408F0A0CE80E439
:1058E000881682E09806A104B10428F4F8016481C6
:1058F000C4018996FBD48FEF481A580A680A780ABF
:105900008FEF881A980AA80AB80A0F5F1F4FE1CFD5
:1059100078941F921FB61F9211248F939F93AF9379
:10592000BF9380915D0390915E03A0915F03B0915E
:1059300060030196A11DB11D80935D0390935E03EA
:10594000A0935F03B0936003BF91AF919F918F913C
:105950001F901FBE1F9018951F920F920FB60F92A7
:1059600011242F933F934F935F936F937F938F9364
:105970009F93AF93BF93EF93FF938091E10082FFDA
:1059800009C08091E20082FF05C08091E1008B7F19
:105990008093E1008091DA0080FF24C08091D800DC
:1059A00080FF20C08091DA008E7F8093DA008091A2
:1059B000D90080FFA9C080E189BD82E189BD09B419
:1059C00000FEFDCF81E080936A0680914C03811137
:1059D00009C00E949A0E0E944B0E8091E2008460E2
:1059E0008093E2008091E10080FF1AC08091E20084
:1059F00080FF16C08091E2008E7F8093E20080914C
:105A0000E20080618093E2008091D8008062809300
:105A1000D80019BC85E080936A0683E08093750105
:105A20008091E10084FF2FC08091E20084FF2BC0B1
:105A300080E189BD82E189BD09B400FEFDCF80917E
:105A4000D8008F7D8093D8008091E1008F7E809375
:105A5000E1008091E2008F7E8093E2008091E2007D
:105A600081608093E20080914B03811509F452C05C
:105A700084E080936A0680916A06843009F052C0FF
:105A800082E0809375018091E10083FF2CC08091BA
:105A9000E20083FF28C08091E100877F8093E100CE
:105AA00082E080936A0610924B038091E1008E7F22
:105AB0008093E1008091E2008E7F8093E2008091EC
:105AC000E20080618093E20042E060E080E00E94BA
:105AD000CB0D8091F00088608093F00081E080938E
:105AE000750180937401FF91EF91BF91AF919F91E8
:105AF0008F917F916F915F914F913F912F910F9077
:105B00000FBE0F901F90189519BC10926A06109244
:105B10004C0368CF8091E30087FF02C083E0A9CFE8
:105B200081E0A7CF81E0ADCF1F920F920FB60F9209
:105B300011241F932F933F934F935F936F937F9302
:105B40008F939F93AF93BF93CF93DF93EF93FF9385
:105B5000E9EEF0E080811091EC008F7010FB1127CE
:105B600017F9182B1082C0EFD0E08881877F8883D7
:105B700078940E944A12E9EEF0E0108288818860F1
:105B800088831F701083FF91EF91DF91CF91BF91B8
:105B9000AF919F918F917F916F915F914F913F91C5
:105BA0002F911F910F900FBE0F901F901895EF929D
:105BB000FF921F93CF93DF93182FEB011092BC003D
:105BC00084EA8093BC000E94A61B7C018091BC00EB
:105BD00087FF26C08091B900887F883029F08091A6
:105BE000B900887F803189F51093BB0084E88093E9
:105BF000BC000E94A61B7C018091BC0087FF1EC0D8
:105C00002091B900287F80E090E0283189F081E080
:105C100090E0203409F480E091958195910908C0C5
:105C2000C7010E94B21BC817D90780F68EEF9FEFFD
:105C3000DF91CF911F91FF90EF900895C7010E94CF
:105C4000B21BC817D907C0F6F1CF8FEF9FEFF0CF87
:105C50001092B9008CE08093B80008950F931F93C1
:105C6000CF93DF93EB018093BB0084E88093BC006B
:105C70000E94A61B8C018091BC0087FF10C0209160
:105C8000B900287F81E090E0283209F480E0919506
:105C900081959109DF91CF911F910F910895CF3F89
:105CA000DC0749F3C8010E94B21BC817D90718F7CF
:105CB0008EEF9FEFEFCFA0E0B0E0E0E6FEE295C20E
:105CC000982E862E772E6A0179010E94A61B5C0110
:105CD00084E1E816F10410F18FEFE816FE0409F1F3
:105CE000C70164E170E068D2162F072F612F702F73
:105CF000892D5DDFEC01892BB1F4082D172DC00E25
:105D0000D11E0C151D0511F02097C1F084E9809378
:105D1000BC00CE01CDB7DEB7EDE083C211E000E0FC
:105D2000E5CF15E0FCCF8FEFE816FE04F9F2C501D0
:105D30000E94B21BE816F906C8F6DFCFB701F801DA
:105D400081918F018BDFEC01DCCFA0E0B0E0EAEACB
:105D5000FEE24BC2982E862E772E6A0189010E94A0
:105D6000A61B5C010431110500F10F3F100701F182
:105D7000C80164E170E020D2EB01BE01892D17DF7C
:105D80007C01892BB9F4C82DD72DCC0EDD1ECC1586
:105D9000DD0519F0E114F104B9F084E98093BC0049
:105DA000C701CDB7DEB7EDE03CC2C1E0D0E0E5CF42
:105DB000C5E0FCCF0F3F100701F3C5010E94B21BE5
:105DC00008171907D0F6DFCFFE018491B80146DF2E
:105DD0007C012196DCCFA0E0B0E0E0EFFEE204C25F
:105DE000982E862E742E652E6901E8010E94A61B4E
:105DF0005C010431110508F10F3F100711F1C801D2
:105E000064E170E0D9D1F62EE72E6F2D7E2D892D1D
:105E1000CEDE8C01892BC1F0CF3FDC07B1F3C50189
:105E20000E94B21BC817D90780F784E98093BC0091
:105E3000C801CDB7DEB7EEE0F3C1FF24F394E12C47
:105E4000E4CF85E0F82EFBCFBE01882D07DF8C0163
:105E5000E72CF62CCE0CDF1CEC14FD0431F30115FD
:105E6000110519F7BE01F70181917F01F7DE8C0161
:105E7000F3CF8EE14A9B02C08150E1F74A9BFECFEF
:105E800008955A9880E28A95F1F75A9A0895FC018C
:105E90008BE08A95F1F728E080E090E031E040E186
:105EA0004A95F1F7880F4A9B02C08160932742E030
:105EB0004A95F1F7000040E14A95F1F7215079F752
:105EC00020E12A95F1F729B132E03A95F1F7000087
:105ED00030E13A95F1F731E022FD93272081920FCE
:105EE00090830895A1E0B0E0E7E7FFE285C1198261
:105EF0008C017C01E60EF11CBCDFCE010196C7DFF0
:105F0000F80181938F01EE15FF05B1F781E09981CA
:105F1000911180E02196E6E08BC1529A5A9A089539
:105F200052985A9AEA9AE9E6F0E080818F7C808361
:105F300008956150770B91E001C0990F6A95EAF7D7
:105F4000692F90E021E0611108C0911591F05A9AF3
:105F500080E28A95F1F75A980895362F382339F060
:105F60005A9A922730E23A95F1F76695ECCF5A9813
:105F7000F9CF5A98EDCFFF920F931F93CF93DF93F2
:105F8000EC018C01060F111D8991F82E7ADF68E073
:105F90008F2DCFDFC017D107B9F7CDB7DEB7E5E05A
:105FA00048C11F920F920FB60F9211240F931F93A7
:105FB0002F933F934F935F936F937F938F939F9311
:105FC000AF93BF93EF93FF93CF93DF930F92CDB730
:105FD000DEB719824EDFCE01019659DF082F0695F4
:105FE00006950695282F22952570902F9570920F73
:105FF000292F237096959695920F982797708981EF
:10600000892B09F055C00B3008F052C080E18A9509
:10601000F1F75A9A529A82E08A95F1F700C05A989D
:1060200088E0089F80011124D801AE5DBE4F16960E
:10603000ED91FD911897309791F06091A8027091C1
:10604000A90214962D913D91260F371F15978D911A
:106050009D91680F791F4C9113978C910995F801C8
:10606000EE5DFE4F6381611549F02091A8023091E9
:10607000A90284819581820F931F7DDF02DF80E179
:106080008A95F1F75A9852985A9A80E18A95F1F7D1
:10609000F801EE5DFE4F6081611549F02091A80284
:1060A0003091A90281819281820F931F1BDFE1DE73
:1060B0000F90DF91CF91FF91EF91BF91AF919F91A1
:1060C0008F917F916F915F914F913F912F911F9190
:1060D0000F910F900FBE0F901F9018950F931F9365
:1060E000CF93DF93EC010B970CF05EC0F894529ABB
:1060F0005A9885E08A95F1F700009C2F9695957047
:106100008C2F8570980F892F837096959695292FDF
:1061100093E0CC0FDD1F9A95E1F7280F822F8C2B8F
:10612000082FAFDE00C068E0802F03DF80E18A9592
:10613000F1F752985A9A4A9B30C087E090E04A990A
:106140002EC0FE01EE5DFE4F6381611559F0209176
:10615000A8023091A90284819581820F931FC2DE2B
:106160008115F9F086DE80E28A95F1F75A98529A05
:1061700080E18A95F1F7CE5DDE4F6881611549F0C7
:106180002091A8023091A90289819A81820F931FE0
:10619000F2DE77DE789481E008C000C0CCCF0197B2
:1061A00049F4529A5A9A789480E0DF91CF911F91E6
:1061B0000F91089500C0C3CFAA1BBB1B51E107C0BC
:1061C000AA1FBB1FA617B70710F0A61BB70B881F87
:1061D000991F5A95A9F780959095BC01CD01089516
:1061E0002F923F924F925F926F927F928F929F92E7
:1061F000AF92BF92CF92DF92EF92FF920F931F93D5
:10620000CF93DF93CDB7DEB7CA1BDB0B0FB6F89485
:10621000DEBF0FBECDBF09942A88398848885F84C5
:106220006E847D848C849B84AA84B984C884DF8036
:10623000EE80FD800C811B81AA81B981CE0FD11D1A
:106240000FB6F894DEBF0FBECDBFED010895EE0F7F
:10625000FF1F0590F491E02D09946927962769277F
:106260007827872778270895FB01DC0104C08D91EA
:106270000190801921F441505040C8F7881B990BB8
:106280000895FB01DC0102C001900D924150504085
:10629000D8F70895DC01CB01FC01F999FECF06C0C7
:1062A000F2BDE1BDF89A319600B40D9241505040D4
:1062B000B8F70895F999FECF92BD81BDF89A992754
:1062C00080B50895A8E1B0E042E050E0E5CFDC0100
:1062D000A40FB51F4150504040F0CB01840F951FD3
:1062E0002E9105D041505040D8F70895262FF999A6
:1062F000FECF92BD81BDF89A019700B4021639F025
:106300001FBA20BD0FB6F894FA9AF99A0FBE0895F5
:106310000396272FECDFEADF252FE9DF242FE7CFD5
:106320000196272FE4DFE2CFF894FFCF28134E1316
:1063300054134E135413A213C4135413BE14CB148A
:10634000201949194E19511954195719D519111AEB
:106350004E20B6205620202024205A2028205E20BF
:106360006A203420AF2038206E203C2072209720F5
:10637000402076209E2046207C2084202C206220F5
:10638000302066204A2080208E20A720AD201A20B1
:106390005220BD20F71FFB1FEE1FF31FFF1F03201E
:1063A0000720FF200521E220E6200821EB200D2117
:1063B000F0201221F5201721FA201C21212126216D
:1063C000E220E6200821EB200D21F0201221F5200B
:1063D0001721FA201C21F22AF62A332B452B502BA9
:1063E0005B2B5E2B5E2B5E2BFE2AFE2ACD2BD02B49
:0C63F000D42BFD2B2A2C2D2C2F2C5C2CE8
:1063FC00E10039003700FFFF0300FF0039050132CF
:10640C000D2E1041106D0D461026100021007F221C
:10641C000003000000010000000000000004010067
:10642C00000004050000000000000409000000004A
:10643C000000010D000000000000010E0000000033
:10644C000000010F00000000000009100000000017
:10645C00000001190000000000000C1A00000000F0
:10646C0000000000010020AE11BE11FC1100000064
:10647C0001FF00FF7844226D3B011901AC00910132
:10648C00AA01CA01FF050200181712110A091916F0
:10649C0013100B081A15140F0C07FFFFFF0E0D0637
:1064AC0033322D2C252434312E2B262335302F2A14
:1064BC002722FFFFFF2928215510320D101410261A
:1064CC00323055345F3F552755155504440244135B
:1064DC004425503A3C373223320D3200210321142B
:1064EC002125102A101810070007001800298B10FE
:1064FC00AE0DD014D026AE308B34813F8B278B154C
:10650C008B049C029C139C25903AA437AE23AE0DB1
:10651C00AE00BF03BF14BF25D02AD018D007E007A8
:10652C00E018E0290202020202020104040404043D
:10653C000401010404040404040404040101010220
:10654C000202020202010404040404040101040412
:10655C0004040404040404010101003131295A1B10
:10656C00750A42415345004C4F5745520052414920
:10657C0053450041444A202620464E000072020139
:10658C00010177020102027D020100038302010373
:10659C0000081018181008009406946697C6F4F5B5
:1065AC00F6F73133E200E900EA00B500B600B700B7
:1065BC00CD008301CC008A019201940121022302B7
:1065CC0024022502260227022A02B300B4006F001F
:1065DC0070009F01CB019F02A002E200E900EA00DB
:1065EC00B500B600B700CD008301CC008A01920142
:1065FC0094012102230224022502260227022A02E8
:10660C00B300B4006F0070009F01CB019F02A00289
:00000001FF
